:020000040800F2
:100000001880002069020008A5350008B12E0008FC
:1000100091350008E50B00081D46000800000000AF
:10002000000000000000000000000000313F000858
:10003000752500080000000009370008FD40000891
:10004000830200088302000883020008830200087C
:10005000830200088302000883020008830200086C
:1000600015260008452600085926000883020008C6
:10007000830200088302000883020008830200084C
:10008000830200088302000883020008830200083C
:100090008302000883020008830200088926000802
:1000A000830200088302000883020008830200081C
:1000B00083020008694100088302000883020008E7
:1000C00083020008830200088302000883020008FC
:1000D00083020008830200088302000883020008EC
:1000E00079250008830200088302000883020008C3
:1000F00083020008830200088302000883020008CC
:1001000083020008830200088302000883020008BB
:1001100083020008830200088302000883020008AB
:10012000830200088302000883020008830200089B
:10013000830200088302000883020008830200088B
:10014000830200088302000883020008830200087B
:10015000830200088302000883020008AD42000801
:10016000830200088302000883020008830200085B
:10017000830200088302000883020008830200084B
:10018000830200088302000800F002F800F05CF827
:100190000AA090E8000C82448344AAF10107DA45E2
:1001A00001D100F051F8AFF2090EBAE80F0013F0D8
:1001B000010F18BFFB1A43F0010318478C470000DA
:1001C000AC4700000A444FF0000C10F8013B13F05C
:1001D000070408BF10F8014B1D1108BF10F8015BA0
:1001E000641E05D010F8016B641E01F8016BF9D193
:1001F00013F0080F1EBF10F8014BAD1C0C1B09D1EA
:100200006D1E58BF01F801CBFAD505E014F8016B5B
:1002100001F8016B6D1EF9D59142D6D370470000ED
:100220000023002400250026103A28BF78C1FBD8FF
:10023000520728BF30C148BF0B6070471FB504F09C
:100240007DFB1FBD10B510BD00F018F91146FFF77A
:10025000F5FF04F095FA00F036F903B4FFF7F2FF6A
:1002600003BC00F03BF900000948804709480047FB
:10027000FEE7FEE7FEE7FEE7FEE7FEE7FEE7FEE756
:10028000FEE7FEE704480549054A064B70470000B3
:100290000141000889010008186000201880002032
:1002A000187000201870002010B5431C02E010F8F0
:1002B000011B71B18107FAD14FF0013202C88C1ACB
:1002C0008C4314EAC211F9D0C01A0A0603D0C01E2A
:1002D00010BDC01A10BD0A0401D0801E10BD090255
:1002E000FCD0401E10BD032A40F2308010F0030CF9
:1002F00000F0158011F8013BBCF1020F624498BF79
:1003000011F801CB00F8013B38BF11F8013BA2F115
:10031000040298BF00F801CB38BF00F8013B11F090
:10032000030300F05280083AC0F0088051F8043B03
:10033000083A51F804CBA0E80810F5E7121D5CBF9D
:1003400051F8043B40F8043BAFF30080D20724BFD0
:1003500011F8013B11F801CB48BF11F8012B24BF64
:1003600000F8013B00F801CB48BF00F8012B7047B3
:1003700002F0FF0343EA032242EA024200F002B81D
:100380004FF000020429C0F0128010F0030C00F0BE
:100390005080CCF1040CBCF1020F18BF00F8012B07
:1003A000A8BF20F8022BA1EB0C0100F042B85FEAD5
:1003B000C17C24BF00F8012B00F8012B48BF00F8D6
:1003C000012B704770477047704710B5203AC0F056
:1003D0000B80B1E81850203AA0E81850B1E8185046
:1003E000A0E81850BFF4F5AF5FEA027C24BFB1E883
:1003F0001850A0E8185044BF18C918C0BDE81040F4
:100400005FEA827C24BF51F8043B40F8043B08BFFC
:100410007047D20728BF31F8023B48BF11F8012BC3
:1004200028BF20F8023B48BF00F8012B70474FF06F
:10043000000200B5134694469646203922BFA0E834
:100440000C50A0E80C50B1F12001BFF4F7AF090740
:1004500028BFA0E80C5048BF0CC05DF804EB890031
:1004600028BF40F8042B08BF704748BF20F8022B74
:1004700011F0804F18BF00F8012B7047754600F04F
:1004800029F8AE4605006946534620F00700854628
:1004900018B020B5FFF7F6FEBDE820404FF000068B
:1004A0004FF000074FF000084FF0000B21F007015C
:1004B000AC46ACE8C009ACE8C009ACE8C009ACE89F
:1004C000C0098D4670470446AFF300802046FFF711
:1004D000C4FE000000487047B85F002001491820A2
:1004E000ABBEFEE726000200704770B506460C461C
:1004F000154608E03046721C96B200F007F804F882
:10050000010B681E85B2002DF4D170BD2DE9F041BC
:1005100004460025002702F03FFFA02002F008FF5C
:1005200002F08CFF054605B129E0201202F000FF21
:1005300002F084FF054605B121E02646E11704EBF1
:1005400011610912A4EB0121C8B202F0F1FE02F020
:1005500075FF054605B112E002F01EFFA12002F072
:10056000E7FE02F06BFF054605B108E0002002F04F
:10057000A9FE074602F036FF3846BDE8F08102F0DA
:1005800031FF0020F9E72DE9F04105460C461646FB
:1005900000270CE02178284600F010F80746012FCC
:1005A00002D00020BDE8F081681C85B2641C3000D8
:1005B000A6F101018EB2EDD10120F3E72DE9F04162
:1005C00004460E46002702F0E7FEA02002F0B0FE2F
:1005D00002F034FF0746201202F0AAFE02F02EFFBE
:1005E00007462546E11704EB11610912A4EB01212E
:1005F000C8B202F09DFE02F021FF0746304602F02D
:1006000097FE02F01BFF074602F0ECFE0F2004F0FD
:1006100025F80120BDE8F0811CB502F0FDFD0121A7
:100620001F2003F03FFB0620009001208DF80400FE
:1006300000208DF8060003208DF8050001208DF8BC
:10064000070069462A4802F0A4FA4FF47B40009064
:100650006946284802F09DFA41F60240009069463A
:10066000254802F096FA43F6014000906946234877
:1006700002F08FFA41F21B4000906946204802F0D8
:1006800088FA04211A4802F0FAFA4FF40051194886
:1006900002F0F5FA0121194802F0F1FA4FF4805105
:1006A000164802F0ECFA4FF48051154802F0E7FAD0
:1006B00002210F4802F0E3FA1021114802F0DFFA9C
:1006C000022010490860012100F08EFA0421002068
:1006D00000F08AFA47F6FF7002F0D6F847F6FF708E
:1006E00002F0E8F800F0C0F802F088FC1CBD000041
:1006F000000002400004024000080240000C0240DA
:10070000001002408C0000201CB50121102003F0D5
:10071000C9FA0420009001208DF8040000208DF813
:10072000060003208DF8050001208DF807006946BA
:10073000034802F02EFA012002F050FC1CBD00001C
:100740000010024010B5002440480078012819D15B
:100750003F48006820F0FF003D4908603D48407870
:10076000096808433A49086001213B48007800F0D5
:100770003BFA04213648006800F036FA002033497D
:10078000087001243548007801281AD130480068E3
:1007900020F47F402E4908602E484078096841EADD
:1007A00000202B49086001212B48007800F01CFA3A
:1007B00004212748006800F017FA00202749087034
:1007C00001242748007801281AD12148006820F424
:1007D0007F001F4908601F484078096841EA0040CF
:1007E0001B49086001211C48007800F0FDF9042134
:1007F0001748006800F0F8F9002019490870012432
:100800001848007801281AD11148006820F07F406C
:100810000F4908600F484078096841EA00600C49B8
:10082000086001210C48007800F0DEF90421084836
:10083000006800F0D9F900200A4908700124012C51
:1008400002D1642003F02AFF10BD000090000020B8
:100850009800002003010020940000209100002057
:10086000920000209300002000B585B00820009081
:1008700000208DF8040003208DF8050002208DF87B
:1008800007006946334802F084F94FF40060009095
:100890006946314802F07DF94FF480700090694656
:1008A0002E4802F076F92020009069462C4802F08C
:1008B00070F90121880303F005FA0B21022003F0EF
:1008C00039FB0821032003F035FB0321002003F04E
:1008D00031FB0521042003F02DFB40F62810029087
:1008E00000208DF80C0008208DF80D0001208DF8F7
:1008F0000E0002A801F07EFF09208DF810000120F3
:100900008DF8110000208DF8120001208DF81300E1
:1009100004A802F049FE17208DF8100001208DF880
:1009200011008DF812008DF8130004A802F03CFEAF
:1009300028208DF8100001208DF8110003208DF87B
:10094000120001208DF8130004A802F02DFE05B05E
:1009500000BD00000000024000080240000C024000
:10096000001002402DE9F04F85B004460D461646B2
:10097000277894F80180A078049094F80590A079E5
:10098000E17900EB01201FFA80FA207A617A00EB0E
:1009900001201FFA80FB3946284603F0EBFA8DF858
:1009A00000908DF80350ADF801A001208DF80400EF
:1009B00002AADDE9000102F02FFA03909DF8081069
:1009C000039801F0CDF8ADF801B000208DF80400D7
:1009D00002AADDE9000102F01FFA03909DF8081059
:1009E000039801F0BDF84FF4FA40ADF80100022081
:1009F0008DF8040002AADDE9000102F00DFA03906F
:100A00009DF80810039801F0ABF82A4641460020F3
:100A100001F0D2FC0021304600F0ACF8002004992F
:100A200001F032FC2946304600F0A4F8002130469F
:100A300000F0A0F805B0BDE8F08F0146162901DAF4
:100A400000207047A1F10A000C2290FBF2F302FB98
:100A5000130008B10020F4E70120F2E77EB5044658
:100A60000D4660788DF80700E0788DF80800207951
:100A70008DF8090060798DF80600A07AE17A00EB24
:100A8000012080B2ADF80400002000906A46DDE944
:100A9000010102F0F7F8064606B97EBD681EC100E6
:100AA000009888400349096808430249086000BF6C
:100AB000F3E7000088000020FEB504460D46164608
:100AC00060788DF80700E0788DF8080020798DF8BF
:100AD000090060798DF80600A07AE17A00EB012028
:100AE00080B2ADF80400002000906A46DDE9010103
:100AF00002F0C8F8074607B9FEBD009840EAC610E4
:100B00000090681EC10000988840034909680843A6
:100B10000149086000BFEFE7880000202DE9F0419F
:100B200005466F781248006800F0004010490860E0
:100B30000026002410E047FA04F000F0010050B154
:100B4000621CD1B206EB4603AA1C02EB8300FFF73E
:100B500085FF701CC6B2641C042CECDB0421044825
:100B6000006800F041F8022003F078FDBDE8F08154
:100B7000880000202DE9F04705460E4695F80180D3
:100B80001748006800F0004015490860002700245D
:100B900019E048FA04F000F0010098B1601C8642A8
:100BA00001D1012000E000208146621CD1B207EB98
:100BB0004703AA1C02EB83004A46FFF77DFF781C1F
:100BC000C7B200BF641C042CE3DB042104480068A6
:100BD00000F00AF8022003F061FDBDE8F087000094
:100BE0008800002000BFFEE7F0B587B004460E463F
:100BF000002500273E4805904FF40040ADF818004E
:100C00003C4803908014ADF81000394801904FF42F
:100C10008040ADF80800012E2BD100BF26E004F083
:100C2000800747B1BDF81010039802F028F80120A2
:100C300003F034FD07E0BDF81010039802F01DF832
:100C4000012003F02BFDBDF80810019802F017F801
:100C5000012003F023FDBDF80810019802F00DF803
:100C6000012003F01BFD6400681CC5B2082DD6DB13
:100C70003CE0042E3AD1002526E004F0004747B1BD
:100C8000BDF81010039801F0FAFF012003F006FDF3
:100C900007E0BDF81010039801F0EFFF012003F00A
:100CA000FDFCBDF80810019801F0E9FF012003F0F8
:100CB000F5FCBDF80810019801F0DFFF012003F0FA
:100CC000EDFC6400681CC5B2202DD6DBBDF8181001
:100CD000059801F0D4FF012003F0E0FCBDF81810E6
:100CE000059801F0CAFF012003F0D8FC07B0F0BD61
:100CF00000040240000802402DE9F04106460F467C
:100D000090461C4601257720044908702246294652
:100D1000012003F09DFBBDE8F0810000B4460020F7
:100D20002DE9F05F81468A4693461E468127394663
:100D30003448FFF725FB02F0B7F804462078314924
:100D4000087060784870A0788870002005E0211D48
:100D50000A5CC11C2B4B5A54401C0E28F7DB04F1D3
:100D60001200FFF7A1FA0546102D01DD102000E06A
:100D700028460546002007E004F112010A5C00F154
:100D80001101204B5A54401CA842F5DB04F122000B
:100D9000FFF78AFA0546202D01DD202000E02846D5
:100DA0000546002007E004F122010A5C00F1210160
:100DB000144B5A54401CA842F5DB04F14200FFF7E3
:100DC00073FA0546402D01DD402000E02846054627
:100DD000002007E004F142010A5C00F14101094BE7
:100DE0005A54401CA842F5DB074B3A4605490320FC
:100DF00000F01AFD804632463946022003F028FBF7
:100E0000BDE8F09FB4460020B44E00202DE9F04F1D
:100E1000A9B081468A4693461E4681273946364800
:100E2000FFF7AEFA684603F085FC6C46207832493D
:100E3000087060784870A0788870002005E0211D57
:100E40000A5CC11C2C4B5A54401C0E28F7DB04F1E1
:100E50001200FFF729FA0546102D01DD102000E0F1
:100E600028460546002007E004F112010A5C00F163
:100E70001101214B5A54401CA842F5DB04F1220019
:100E8000FFF712FA0546202D01DD202000E028465C
:100E90000546002007E004F122010A5C00F121016F
:100EA000154B5A54401CA842F5DB04F14200FFF7F1
:100EB000FBF90546402D01DD402000E028460546AF
:100EC000002007E004F142010A5C00F141010A4BF5
:100ED0005A54401CA842F5DB084B3A460649032009
:100EE00000F0A2FC804632463946032003F0B0FAF7
:100EF00029B0BDE8F08F0000B4460020B44E0020B9
:100F00002DE9F041AAB006460F4690461C460E2534
:100F100001A803F00FFC2A460DF18E010548FFF7EA
:100F2000E2F922462946042003F092FA2AB0BDE8ED
:100F3000F0810000B446002003F010FC012080F393
:100F4000138800BF00BFBFF34F8F0748006800F44D
:100F5000E06006490843001D03490860BFF34F8F56
:100F600000BF00BFFEE700000CED00E00000FA0546
:100F70002DE9F04105460C461646984627465EB1D7
:100F80002146284601F0D0FF08B9BDE8F08120468F
:100F900004EBD071C1F34F07142F07DA002003E0F0
:100FA000295C034A1154401CB842F9DB00BFECE74E
:100FB000200100202DE9F04106460F4690461C46D0
:100FC00014252A4605490648FFF78DF92246294689
:100FD000072003F03DFABDE8F08100002001002069
:100FE000B44600202DE9F043A9B005460C4616464C
:100FF0009946012704F0FF0856B1204604EBD07152
:10100000C1F347082146284601F08EFF00B90027AA
:10101000B8F10E0F00DA002767B1684603F08AFBCB
:101020000E2229460DF18A00FFF75DF9684603F0AC
:101030008BFB03E00121022000F0AAFC29B0BDE8EF
:10104000F0832DE9F04104460D4616461F46012166
:10105000902000F09DFCBDE8F08170472DE9FF4F26
:1010600087B004460E465048007810B10BB0BDE87A
:10107000F08F01204C490870324621464B48FFF75B
:1010800032F93046FFF7D9FC38B9002046490870DC
:101090000121052000F07CFCE8E7A6F10800C5B2BC
:1010A000281D00F0FF08615D681C205C01EB002139
:1010B000A81C205C01EB0041E81C205C01EB0060F7
:1010C000069014F8081008F10100205C01EB0020E4
:1010D00080B205902946204601F010FF0490294671
:1010E000204601F06EFF814604990698884202D19D
:1010F0000598484507D000202B4908700121FF20A2
:1011000000F046FCB2E74FF0000A207800F0010042
:101110000390607800F00F0002902046FFF7FEFC7D
:1011200000271AE00298384100F0010B791CC8B280
:10113000594602F0EBFABBF1000F0DD07A1CD1B288
:101140000AEB4A03A21C02EB83002246FFF70AFCCB
:101150000AF1010000F0FF0A7F1C042FE2DB039874
:1011600028B94FF40061124801F089FD04E04FF402
:1011700000610F4801F081FD02200190002006E08F
:10118000B11E0144615C0B4A1154411CC8B20228D3
:10119000F6DB22200A9A019903F05AF9002002494D
:1011A000087000BF62E70000840000207C5F002020
:1011B000000C0240B44600202DE9F0470546884661
:1011C00091469A464A464146284601F0D9FB28B93D
:1011D0000121052000F0DCFBBDE8F0872F78002618
:1011E00000240FE047FA04F000F0010048B1621C4F
:1011F000D1B206EBC6036A1C981801F071FB701C93
:10120000C6B2641C042CEDDB00BFE5E72DE9F04716
:101210000546884691469A462E780027002420E00D
:1012200046FA04F000F00100D0B1012000EB840088
:10123000285C00F00101022000EB8400285C61F3CF
:101240005F10074632463946042001F0B5F8042005
:1012500000EB84002F5C32463946052001F0ACF8E3
:10126000641C042CDCDB00F0A1FBBDE8F08700006F
:101270002DE9F0478046894692461D4608261348C8
:10128000008884B2200A124908704C701148008806
:1012900084B2200A8870CC700F48008884B2200A7B
:1012A00008714C710D48008884B2200A8871CC7195
:1012B0000B4B3246302000F0B7FA07462A4631463B
:1012C000302003F0C5F8BDE8F0870000BC00002026
:1012D000B4460020BE000020C0000020C200002054
:1012E000B44E00202DE9F04105460E4617461C4637
:1012F0002146012002F05EFFBDE8F0812DE9F041BA
:1013000004460D4616461F460121902000F040FB82
:10131000BDE8F0812DE9F05F07460C4615461E46F4
:101320004FF0010804F0FF095DB1204604EBD071D5
:10133000C1F347092146384601F0F6FD08B94FF0E0
:101340000008B9F1010F01D04FF00008B8F1000F0B
:1013500005D10121052000F01BFBBDE8F09F4FF0F7
:10136000640A0749384602F00DFA824602F0A1F9F4
:10137000834632465146332003F06AF800BFECE75B
:10138000B44600202DE9F04104460E461546984625
:1013900001272B463A463146204601F0E8FD28B9A0
:1013A0000121022000F0F4FABDE8F081207802F07B
:1013B00047FC00BFF8E700002DE9F05F06460C4649
:1013C00017469B464FF0010804F0FF095FB1204625
:1013D00004EBD071C1F347092146304601F0A4FD6A
:1013E00008B94FF00008B9F1050F01DA4FF0000815
:1013F000B8F1000F17D096F800A001200D49087031
:1014000000250DE04AFA05F000F0010038B1681C33
:10141000C1B2701C00F0E0F90A2003F03FF96D1C26
:10142000042DEFDB03E00121052000F0B1FABDE857
:10143000F09F0000840000202DE9F05F06460C4676
:1014400017469B464FF0010904F0FF0A5FB12046A2
:1014500004EBD071C1F3470A2146304601F064FD28
:1014600008B94FF00009BAF1050F01DA4FF0000991
:10147000B9F1000F1ED0012004E0315C01EB082817
:10148000411CC8B20528F8DB3078801FC5B225B9E9
:101490000121404600F064FB05E0012D03D102214B
:1014A000404600F05DFB022D03D10321404600F0D1
:1014B00057FB03E00121052000F06AFABDE8F09F28
:1014C0002DE9F05F06460D4617469B464FF0010991
:1014D00005F0FF0A5FB1284605EBD071C1F3470A5A
:1014E0002946304601F020FD08B94FF00009BAF155
:1014F000020F01DA4FF00009B9F1000F05D1012107
:10150000052000F045FABDE8F09F96F80180347898
:10151000012C05D101224146022000F04DFF16E0CA
:10152000022C05D102224146104600F045FF0EE094
:10153000042C05D103224146022000F03DFF06E0C5
:10154000082C04D104224146022000F035FF14206B
:1015500003F0A4F800BFD6E72DE9F047044688461B
:10156000174699463B4606224146204601F0FFFCBD
:1015700028B90121052000F00BFABDE8F08760785A
:10158000217800EB01260025022004E0215C01EB1C
:101590000525411CC8B20628F8DB07490E7007482C
:1015A000056001213046FFF71FFB04212846FFF7A5
:1015B0001BFB00BFE1E70000940000209800002022
:1015C0002DE9F04105460E4614461F4623461222D9
:1015D0003146284601F0CBFC28B90121052000F056
:1015E000D7F9BDE8F0811221284601F05DFF00BF68
:1015F000F7E700002DE9F0479AB006460C4617467B
:101600009A464FF0010804F0FF094FB1204604EB61
:10161000D071C1F347092146304601F085FC804670
:10162000B9F1070F01DA4FF00008B8F1000F06D149
:101630000121052000F0ACF91AB0BDE8F08716488A
:10164000007800B1F8E7012013490870652C0ADA28
:10165000002004E0FF2122180DF80210401CC4F104
:1016600065018142F6DC224631466846FEF73BFEC4
:101670000DF10101684602F0DAF80546012D02D1AC
:1016800000F094F903E00121FF2000F081F900202F
:101690000149087000BFCFE7840000202DE9F04128
:1016A00004460D4616461F4602F0D2FDBDE8F08105
:1016B000F8B504460D4616461F4600F077F903F0CC
:1016C000C1F800200090F8BD00F070F900BFFEE7FF
:1016D0002DE9F04705460C46174698464FF001099C
:1016E00004F0FF0A5FB1204604EBD071C1F3470A52
:1016F0002146284601F018FC08B94FF00009BAF15C
:10170000020F01DA4FF00009B9F1000F05D10121F4
:10171000052000F03DF9BDE8F0870226287820B1C9
:10172000012804D0022806D103E0292604E0082677
:1017300002E0082600E000BF00BF06F10801FF221A
:101740001448FEF715FE287820B1012808D0022899
:1017500016D10DE03A2210490E48FEF7C4FD10E004
:101760000C480E49096801600D490968416008E0AC
:1017700008480C49096801600B490968416000E0AC
:1017800000BF00BF42463146E32002F061FE00BFC9
:10179000C1E70000B44600207C5F00201801002053
:1017A0001C010020A8020020A40200202DE9F04125
:1017B00004460F4690461D46802680222146054855
:1017C000FEF791FD2A463146E42002F041FEBDE8D5
:1017D000F0810000B44600202DE9FE4304460D468A
:1017E00026786778A078E17800EB01201FFA80F86E
:1017F0000EB9012600E000268DF800708DF8035028
:10180000ADF801808DF8046002AADDE9000101F065
:1018100003FB81469DF80810484600F0D5F80120EA
:1018200002F01CFFBDE8FE832DE9F04106460F469D
:1018300015461C4655202070AA206070BB20A07061
:10184000E6702571280A6071002D04DD2A463946AC
:10185000A01DFEF748FD0D21A81D21540A21E81DF9
:101860002154401CBDE8F0812DE9F0413A483B4944
:10187000097830F811604FF6FF70864200D15FE0C2
:101880004FF6FF703449354A127821F812000020D3
:101890000CE03349895D334A1154711C44F208024B
:1018A00091FBF2F302FB13118EB2401CB0F5026FF4
:1018B000EFDB2C480078552807D12A484078AA2821
:1018C00003D128488078BB2800D039E0254DA8886E
:1018D000801D2946085C0D2804D1A888C01D085C1D
:1018E0000A2800D02CE01C481C49097830F8116007
:1018F0001C4F002420E004EB44001B4911F8200099
:10190000F978884216D104EB4400DFF85C8008EBDC
:101910008000437A04EB440008EB8000027AB98827
:1019200004EB440008EB8000D0F804C00D48801D93
:10193000E04703E0601CC4B21E2CDCDB00BF00BF2C
:1019400006480078401C142190FBF1F201FB1200C4
:1019500002490870BDE8F08134570020AD00002036
:10196000AC0600205C5700203401002070B5142420
:101970000125224604490548FEF7B5FC2A462146C2
:10198000072002F065FD70BD20010020B446002054
:1019900070B504460D460126034804702A463146B8
:1019A000B02002F055FD70BDB446002010B50224F1
:1019B000C0200449087048700122214602F048FD09
:1019C00010BD0000B44600202DE9F04186B0044669
:1019D0000D4600260027B0465E480290C014ADF8C0
:1019E0000C005C4800908014ADF80400012D04D078
:1019F000022D08D0032D13D10CE05748049001208C
:101A0000ADF814000DE0534804904FF40050ADF8C9
:101A1000140000BF514804900420ADF8140000BF2A
:101A200000BF00BFBDF81410049801F026F9012092
:101A300002F034FEBDF81410049801F020F90120E2
:101A400002F02CFEBDF81410049801F016F90120E4
:101A500002F024FEBDF80C10029801F010F9BDF858
:101A60000410009801F00BF9012002F017FEBDF8F8
:101A70000C10029801F001F9012002F00FFEBDF8F0
:101A80000410009801F0F9F8012002F007FE00268A
:101A900043E0002725E004F00048B8F1000F05D02E
:101AA000BDF80C10029801F0EAF804E0BDF80C1043
:101AB000029801F0E2F8012002F0F0FDBDF80410F8
:101AC000009801F0DCF8012002F0E8FDBDF80410F8
:101AD000009801F0D2F8022002F0E0FD6400781CCA
:101AE000C7B2082FD7DBBDF80C10029801F0C5F87B
:101AF000012002F0D3FDBDF80410009801F0BFF8FA
:101B0000012002F0CBFDBDF80410009801F0B5F8FB
:101B1000022002F0C3FD701CC6B2042EB9DBBDF872
:101B20000410009801F0ABF8012002F0B7FDBDF8F9
:101B30000C10029801F0A3F8012002F0AFFDBDF8EF
:101B40001410049801F09BF8012002F0A7FD06B0E4
:101B5000BDE8F08100040240000C02400000024099
:101B60002DE9FC4704460D460027C4F3034848F01E
:101B70003009A6B2012D04D0022D09D0032D16D1B3
:101B80000EE01827264800900120ADF8040010E070
:101B90001A27244800904FF40050ADF8040008E0E4
:101BA0001C27214800900420ADF8040001E0BDE8A6
:101BB000FC8700BF01F08CFA384601F055FA01F0BD
:101BC000D3FA00B127E0484601F04EFA01F0CCFA12
:101BD00000B120E0300A01F047FA01F0C5FA00B187
:101BE00019E0F0B201F040FA01F0BEFA00B112E0E3
:101BF00001F094FABDF80410009801F03EF80520B9
:101C000002F04CFDBDF80410009801F038F80120F6
:101C100002F024FDCBE701F081FA00BFC7E7000026
:101C2000000C0240000402400000024070B505466E
:101C30000024022D18D0032D2BD0042D3ED04C486B
:101C4000006820F440104A490860084600680860AF
:101C500004E0601CC4B2012002F020FD4548006889
:101C600008B1C82CF5DB3FE04348006820F4402071
:101C70004149086008460068086004E0601CC4B27E
:101C8000012002F00BFD3D48006808B1C82CF5DBCF
:101C90002AE03B48006820F44020394908600846A3
:101CA0000068086004E0601CC4B2012002F0F6FC89
:101CB0003448006808B1C82CF5DB15E02C480068F2
:101CC00020F003002A49086008460068086004E024
:101CD000601CC4B2012002F0E1FC264828380068EC
:101CE00008B1C82CF4DB00BF00BFC82C01DB012009
:101CF00070BD0024022D0FD0032D19D0042D23D048
:101D000004E0601CC4B2012002F0C8FC194800685D
:101D100008B9F02CF5DB24E004E0601CC4B201201B
:101D200002F0BCFC1548006808B9F02CF5DB18E09F
:101D300004E0601CC4B2012002F0B0FC114800684D
:101D400008B9F02CF5DB0CE004E0601CC4B2012003
:101D500002F0A4FC07482838006808B9F02CF4DB2E
:101D600000BF00BFF02C01DB0120C1E70020BFE76E
:101D70000008024028024142000C024024824142F5
:101D8000001002402402424210B5002400F0E6F99F
:101D900000F08AF90120FFF749FF0220FFF746FF14
:101DA0000320FFF743FF0420FFF740FFCC2000F0A3
:101DB000EBF9BE2000F0E8F9012000F07FF804B252
:101DC000200104B22046E11704EB11710C111548F3
:101DD0000480022000F072F804B2200104B2204610
:101DE000E11704EB11710C110F480480032000F07F
:101DF00065F804B2200104B22046E11704EB11712A
:101E00000C110A480480042000F058F804B22001A4
:101E100004B22046E11704EB11710C110448048050
:101E2000204610BDBC000020BE000020C0000020E5
:101E3000C20000201CB540F20140009001208DF846
:101E4000040000208DF8060002208DF80500012016
:101E50008DF807006946164800F09BFE4FF40070AD
:101E600000906946134800F094FE4FF40070009013
:101E70006946114800F08DFE00F016F90120FFF7C9
:101E8000D5FE012801D000201CBD0220FFF7CEFEA8
:101E9000012801D00020F7E70320FFF7C7FE012843
:101EA00001D00020F0E70420FFF7C0FEECE70000BF
:101EB00000080240000C0240001002402DE9F041F1
:101EC0000446002600251AE0022C03D100F050F849
:101ED00007460EE0032C03D100F07EF8074608E029
:101EE000042C03D100F0ACF8074602E000F00CF837
:101EF000074607FA05F0304386B2681CC5B20C2DC0
:101F0000E2DB3046BDE8F08110B5002415480068DA
:101F100020F44010134908600846006840F480101F
:101F20000860002010490860022002F0B7FB012081
:101F30000E49C1F8A8020B48006820F44010094976
:101F400008600846006808600C2002F0A7FB0648FD
:101F50008038006800B10124322002F09FFB204647
:101F600010BD000000080240A802414200004142AA
:101F700010B500241548006820F44020134908607B
:101F80000846006840F4802008600020104908607E
:101F9000022002F083FB01200E49C1F8A4020B4885
:101FA000006820F44020094908600846006808607D
:101FB0000C2002F073FB06488038006800B1012451
:101FC000322002F06BFB204610BD0000000C0240E6
:101FD000A48241420080414210B5002415480068A7
:101FE00020F44020134908600846006840F480202F
:101FF0000860002010490860022002F04FFB012019
:102000000E49C1F8A4020B48006820F44020094999
:1020100008600846006808600C2002F03FFB064894
:102020008038006800B10124322002F037FB2046DE
:1020300010BD000000100240A402424200004242D3
:1020400010B500241548006820F00300134908600B
:102050000846006840F00100086000201049086050
:10206000022002F01BFB01200E49C1F880020B4840
:10207000006820F00300094908600846006808600D
:102080000C2002F00BFB06488038006800B10124E8
:10209000322002F003FB204610BD00000008024081
:1020A000800241420000414210B52448006820F4FB
:1020B0004010224908600846006840F4801008601B
:1020C0001F48006820F440201D4908600846006849
:1020D00040F4802008601B48006820F44020194923
:1020E00008600846006840F48020086013480068D3
:1020F00020F00300114908600846006840F0010024
:1021000008600020104908601049C1F8A402104975
:1021100008601049C1F8800240F2EE2002F0BEFAD9
:102120000120094908600C4908600949086009490B
:10213000C1F880020F2002F0B1FA10BD0008024081
:10214000000C024000100240A802414200804142BF
:10215000A402424200004142A482414210B5FFF76E
:10216000A3FF0120FFF762FD0220FFF75FFD0320C0
:10217000FFF75CFD0420FFF759FDCC2000F004F8C8
:10218000442000F001F810BD70B5044636480068E0
:1021900020F44010344908600846006840F480107C
:1021A00008603248006820F4402030490860084642
:1021B000006840F4802008602D48006820F440202A
:1021C0002B4908600846006840F4802008602648D3
:1021D000006820F00300244908600846006840F0C9
:1021E0000100086001253CE004F001066410DEB146
:1021F0000020204908602049C1F8A4021F49086056
:102200001F49C1F88002022002F048FA0120194952
:1022100008601C490860194908601949C1F8800222
:102220003C2002F03BFA1AE00020124908601249F3
:10223000C1F8A402114908601149C1F880023C208C
:1022400002F02CFA01200B4908600E4908600B4986
:1022500008600B49C1F88002022002F01FFA681CD6
:10226000C5B2082DC0DD70BD00080240000C024060
:1022700000100240A802414200804142A4024242B2
:1022800000004142A48241422DE9FF4106460D462D
:102290000024374647480290C014ADF80C0045486A
:1022A00000904FF40050ADF80400002F56D000BF4E
:1022B00026E007F08008B8F1800F05D1BDF80C10BA
:1022C000029800F0DCFC04E0BDF80C10029800F06D
:1022D000D4FC022002F0E2F9BDF80410009800F0EE
:1022E000CEFC022002F0DAF9BDF80410009800F0EC
:1022F000C4FC022002F0D2F97806070E601CC4B2BA
:10230000082CD6DB002426E005F08008B8F1800F09
:1023100005D1BDF80C10029800F0B1FC04E0BDF846
:102320000C10029800F0A9FC022002F0B7F9BDF8E9
:102330000410009800F0A3FC022002F0AFF9BDF8F1
:102340000410009800F099FC022002F0A7F968063A
:10235000050E601CC4B2082CD6DB29E0002425E061
:1023600005F00108B8F1000F05D0BDF80C10029877
:1023700000F085FC04E0BDF80C10029800F07DFC34
:10238000022002F08BF9BDF80410009800F077FCF1
:10239000022002F083F9BDF80410009800F06DFCF3
:1023A000022002F07BF96D10601CC4B2082CD7DB50
:1023B000BDE8FF81000C02402DE9F04387B00746DD
:1023C0000D46904600243E4667480390C014ADF881
:1023D0001000654801904FF40050ADF80800B8F1C6
:1023E000010F09D0B8F1020F0CD0B8F1030F0FD0D4
:1023F000B8F1040F18D111E05B4805908014ADF8D6
:10240000180012E0594805908014ADF818000CE04F
:10241000574805900220ADF8180006E05348059093
:102420001020ADF8180000E000BF00BFBDF8181084
:10243000059800F022FC022002F030F9002E56D060
:10244000002426E006F08009B9F1800F05D1BDF81F
:102450001010039800F013FC04E0BDF8101003986E
:1024600000F00BFC022002F019F9BDF808100198E9
:1024700000F005FC022002F011F9BDF808100198E7
:1024800000F0FBFB022002F009F97006060E601C4A
:10249000C4B2082CD6DB002426E005F08009B9F18F
:1024A000800F05D1BDF81010039800F0E8FB04E0A0
:1024B000BDF81010039800F0E0FB022002F0EEF8E7
:1024C000BDF80810019800F0DAFB022002F0E6F8EF
:1024D000BDF80810019800F0D0FB022002F0DEF8F1
:1024E0006806050E601CC4B2082CD6DB29E0002467
:1024F00025E005F00109B9F1000F05D0BDF8101075
:10250000039800F0BCFB04E0BDF81010039800F045
:10251000B4FB022002F0C2F8BDF80810019800F0E8
:10252000AEFB022002F0BAF8BDF80810019800F0E6
:10253000A4FB022002F0B2F86D10601CC4B2082C9B
:10254000D7DBBDF81810059800F099FB022002F0C7
:10255000A5F8BDF81810059800F08FFB022002F0D6
:102560009DF807B0BDE8F083000C02400010024067
:10257000000002407047000010B54FF4806000F08A
:102580002DF9012814D1142002F068F84FF400410D
:102590001B4800F069FB30B91A480078012802D1C5
:1025A0000020184908704FF4806000F011F925E010
:1025B0004FF4805000F012F9012814D1142002F0D9
:1025C0004DF84FF48051104800F04EFB30B90F48E1
:1025D0000078012802D100200C4908704FF4805087
:1025E00000F0F6F80AE04FF4006000F0F7F8012878
:1025F00004D107490870C00200F0EAF810BD0000DD
:10260000000C0240A900002000000240A8000020A9
:102610009000002010B5142002F020F80421074893
:1026200000F022FB30B906480078012802D10020D2
:1026300003490870042000F0CBF810BD000C0240E4
:10264000A700002010B5012002490870082000F002
:10265000BFF810BD9200002010B5142001F0FEFF5D
:102660001021074800F000FB30B906480078012827
:1026700002D1002003490870102000F0A9F810BD15
:10268000000C0240A600002010B5402000F0A6F883
:10269000012812D1142001F0E1FF4021124800F07E
:1026A000E3FA30B911480078012802D100200F491F
:1026B0000870402000F08CF815E0202000F08EF823
:1026C000012805D10A490870202000F081F80AE0AD
:1026D0004FF4807000F082F8012804D10549087099
:1026E000000200F075F810BD000C0240A5000020AB
:1026F00093000020910000200EB50121880301F015
:10270000E1FA0221032001F015FC0421032001F06D
:1027100011FC0621032001F00DFC0821032001F02B
:1027200009FC0A21002001F005FC0C21002001F029
:1027300001FC0521042001F0FDFB41F274500090E2
:1027400000208DF8040008208DF8050001208DF888
:102750000600684600F04EF808208DF808000120B9
:102760008DF8090002208DF80A0001208DF80B0079
:1027700002A800F019FF0A208DF8080002208DF849
:10278000090001208DF80A008DF80B0002A800F066
:102790000BFF28208DF8080003208DF80900022087
:1027A0008DF80A0001208DF80B0002A800F0FCFE55
:1027B00017208DF8080004208DF8090002208DF8FC
:1027C0000A0001208DF80B0002A800F0EDFE0EBDFE
:1027D0000149086070470000143C01400146002098
:1027E000034A12680A400AB1012000E00020704745
:1027F000143C0140002123498279002A3AD00A463C
:10280000126803689A430B461A600A1D126803682F
:102810009A430B1D1A60027911440A6803681A432F
:102820000A60184A0832126803689A43154B083345
:102830001A601A1D126803689A43124B0C331A600F
:102840004279102A0ED11A1F126803681A430D4BE1
:1028500008331A601A1D126803681A43094B0C33B7
:102860001A600DE00749427911440A6803681A4367
:102870000A6005E0027911440A6803689A430A6015
:1028800070470000003C01402DE9F041054602265A
:102890000C274FF00108064C44EA076444EA084458
:1028A0002C4331462046FFF78FF8BDE8F081000049
:1028B000000030102DE9F041054602260C274FF0AC
:1028C0000308064C44EA076444EA08442C433146B2
:1028D0002046FFF779F8BDE8F081000000003010D5
:1028E0002DE9FF5F04466578A678E77894F80880BC
:1028F0002079617900EB01201FFA80F9A079E17954
:1029000000EB01201FFA80FA00201B4908601B48D9
:1029100000680190002000908DF80C508DF80D603B
:102920008DF80A708DF80E806B4601AADDE9020170
:1029300000F02AFA8346BBF1000F01D1BDE8FF9FEA
:102940009DF800000C4908600C49019808600121BD
:1029500009480068FEF748F9042108480068FEF7B6
:1029600043F94846FFF7A6FF5046FFF78DFF0220C8
:1029700001F074FE00BFE1E78C0000208800002019
:102980002DE9F04106460D4617460B2D02DA0020D0
:10299000BDE8F0810024002009E001218140327867
:1029A0001140012901D1611CCCB2411CC8B20428DC
:1029B000F3DBA81E04EBC401884201D00020E7E746
:1029C0004FB104EBC400801C00F0FF0841463046C4
:1029D00000F0AAFADCE70120DAE70000014908600C
:1029E000704700000C3C024030B10749096841F4CF
:1029F0008061054A116005E00349096821F480619E
:102A0000014A116070470000003C024070B5044666
:102A10000A460026092502B909E0012A01D1160259
:102A200005E0022A01D1160201E04FF4407600F0E1
:102A30009FF80546092D28D11548006820F44070FC
:102A4000134908600846006830430860084600687B
:102A500020F0F80008600846006844F002010843CE
:102A60000B4908600846006840F48030086000F0B8
:102A70007FF805460648006820F002000449086017
:102A80000846006820F0F8000860284670BD000085
:102A9000103C024009201349096801F48031B1F566
:102AA000803F01D101201CE00E49096801F01001AE
:102AB00009B1062015E00B49096801F4807109B1DC
:102AC00002200EE00749096801F0EF0109B1072073
:102AD00007E00449096801F0020109B1082000E09B
:102AE000092070470C3C02400348006840F0004059
:102AF0000149086070470000103C024030B50246B2
:102B00000C46092500F034F80546092D19D10E4868
:102B1000006820F440700C4908600846006840F4E2
:102B2000007008600846006840F00100086014600A
:102B300000F01EF805460448006820F00100024934
:102B40000860284630BD0000103C0240054800687F
:102B500000F0004028B1044802490C3908600348DD
:102B600008607047103C024023016745AB89EFCDF8
:102B700008B509200090FFF78DFF009002E0FFF7F5
:102B800089FF00909DF800000128F8D09DF8000012
:102B900008BDF0B50A4600210023002400BF3DE037
:102BA000012505FA01F3156805EA03049C4234D1B6
:102BB00005684F000326BE40B543056015794E00F9
:102BC000B5400668354305601579012D02D01579A9
:102BD000022D16D185684F000326BE40B54385609F
:102BE00055794E00B54086683543856045680126B5
:102BF0008E40B5434560456896798E40B6B2354300
:102C00004560C5684F000326BE40B543C560D57911
:102C10004E00B540C6683543C560491C1029BFD376
:102C2000F0BDF0B5002300244D07ED0E02FA05F3C8
:102C3000CE1000F1200555F826504E07F70E0F264E
:102C4000BE40B543CF1000F1200646F82750CE1005
:102C500000F1200555F8265045EA0304CE1000F196
:102C6000200545F82640F0BD0246002013690B40C0
:102C70000BB1012000E000207047418370470183C1
:102C80007047000017B500210023BDF800004FF683
:102C9000FF74A04200D117E0BDF80000B0F5FA7F44
:102CA00002D141F005010FE0BDF80000C82802D1B3
:102CB00041F0010108E0BDF80000142802D141F004
:102CC000030101E000201EBD9DF8050038B99DF804
:102CD0000200012803D12B480078014318E09DF839
:102CE000050038B99DF8020020B926484078014314
:102CF00001230DE09DF80500012807D19DF8020091
:102D000020B9204880780143012301E00020DAE760
:102D1000D3B19DF8040010B941F030012FE09DF8C7
:102D200004000C2802D141F0100128E09DF80400B5
:102D30001A2802D141F0200121E09DF80400262844
:102D400000D11CE00020BEE79DF8040000B916E0A9
:102D50009DF80400062802D141F010010FE09DF813
:102D600004000C2802D141F0200108E09DF8040085
:102D7000142802D141F0300101E00020A3E71160E6
:102D80000120A0E7000100200FB502219DF80600F8
:102D900000F0010008B141F080019DF8050000B984
:102DA0001BE09DF80500012802D141F0080114E064
:102DB0009DF80500022804D1106840F00040106022
:102DC0000BE09DF80500032804D1106880F0004056
:102DD000106002E0002004B000BD9DF80200012850
:102DE00002D141F0400105E09DF8020000B901E088
:102DF0000020F0E79DF80400012800D108E09DF8CC
:102E00000400052802D141F0200101E00020E2E7A2
:102E100019700120DFE7000077B5214800219DF8F7
:102E200004503DB99DF800500DB9042500E003257C
:102E300029460AE09DF80450012D06D19DF8005066
:102E40000DB9022500E0012529469DF803506D1EAD
:102E5000C5EB0515134E354401EB4106AD5D6D1F05
:102E600015709DF803506D1EC5EB05150D4E3544CC
:102E700001EB41063544AC789DF803506D1EC5EB5F
:102E80000515084E354401EB410635446B7840EAA0
:102E9000046040EA0340BDF8015028437EBD0000B5
:102EA00000003010C40000200048704700000020DF
:102EB00002480349086000BFFEE700000400FA056D
:102EC0000CED00E0002111E00846082208E000F0C7
:102ED00001031BB1074B83EA500000E04008521E7B
:102EE000002AF4DC044B43F82100491CFF29EBDDE8
:102EF000704700002083B8EDAC02002030B50246D8
:102F00000B464FF0FF31002008E0CCB2155C6C405E
:102F1000044D55F8244084EA1121401C9842F4D312
:102F2000C84330BDAC02002030B5034609B90120CA
:102F300030BD084601EBD0725210A1EB42020AB13B
:102F40000020F5E7084601EBD072C2F34F040022DF
:102F500009E0985CC043C0B215195D5DA84201D07C
:102F60000020E5E7521CA242F3DB0120E0E72DE957
:102F7000F04381460C4615461E4614B90120BDE8B3
:102F8000F083012704F0FF0856B1204604EBD0710E
:102F9000C1F3470821464846FFF7C6FF00B900279E
:102FA000A84500D000273846E9E710B502460020C2
:102FB00004E0135CDB4344181355401C8842F8DBE3
:102FC00010BD10B502460023002003E0145C1C4431
:102FD000A3B2401C8842F9D3184610BD10B5044670
:102FE000012C04D104210448FFF749FE03E0042129
:102FF0000148FFF742FE10BD001002401CB5012140
:10300000022000F04FFE4FF4C050009001208DF8D8
:10301000040000208DF8060003208DF80500012033
:103020008DF8070069460B48FFF7B3FD01200A49F8
:1030300008600A49C1F8AC0201210948FFF71FFEE8
:103040004FF400510348FFF71AFE04210548FFF72B
:1030500016FE1CBD00040240B08240420080404287
:10306000000C02400000024070B50446154800689C
:1030700020F44000134908600846006840F48000CE
:103080000860002010490860002517E0E0090E499B
:10309000091F08606006040E022001F0FFFA0120FB
:1030A0000A49C1F8B002022001F0F8FA00200649EE
:1030B0000860022001F0F2FA681CC5B2082DE5DBB9
:1030C00070BD000000040240B082404200804042D7
:1030D00010B50F48006820F440000D49086008460C
:1030E000006840F48000086001200A4908600A492D
:1030F000C1F8B002042001F0D1FA002005490860AF
:10310000042001F0CBFA00200349C1F8B00210BD41
:1031100000040240AC8240420080404210B50F489B
:10312000006820F440000D4908600846006840F43B
:103130008000086000200A4908600A49C1F8AC0212
:10314000042001F0ABFA0120054908600549C1F8E7
:10315000AC02042001F0A2FA10BD000000040240FD
:10316000B08240420080404210B5002413480068FD
:1031700020F44000114908600846006808600120FA
:103180000F49086001F08AFA01200E49C1F8B00227
:1031900001F084FA07E0601CC4B2FA2C03DDFFF7EB
:1031A000BDFF012010BD0648803800680028F2D11C
:1031B0000349091D086000BFF4E700000004024055
:1031C000AC8240420080404210B500200F490860A8
:1031D0000F48006820F440400D4908600846006828
:1031E00040F48040086000200A49C1F89C020A208F
:1031F00001F054FA0120054908600A2001F04EFA56
:1032000000200449C1F8980210BD00009882404295
:1032100000040240008040421CB50121022000F061
:1032200041FDE020009001208DF8040000208DF881
:10323000060003208DF8050000208DF80700694680
:103240000948FFF7A6FC0020084908600A2001F0A1
:1032500025FA01200649C1F894020449091D0860B5
:103260000349C1F89C021CBD000402409482404204
:103270000080404210B500200F4908600F480068E8
:1032800020F440400D4908600846006840F4804042
:10329000086001200A49C1F89C020A2001F0FEF9E9
:1032A0000120054908600A2001F0F8F900200449CE
:1032B000C1F8980210BD000098824042000402400C
:1032C0000080404270B5054600241648006820F48E
:1032D000404014490860084600680860002616E06F
:1032E0000020114908600A2001F0D8F901200F4997
:1032F000C1F898026006040E0B487C38006808B1DB
:10330000601CC4B20A2001F0C9F9701CC6B2082EB4
:10331000E6DB15B9FFF7AEFF01E0FFF755FF2046EA
:1033200070BD00000004024098824042008040428C
:1033300070B504461548006820F440401349086001
:103340000846006840F4804008600020104908608A
:10335000002517E0E0090E49091D08606006040E0B
:103360000A2001F09BF901200A49C1F898020A20BD
:1033700001F094F90020064908600A2001F08EF956
:10338000681CC5B2082DE5DB70BD000000040240DA
:10339000988240420080404210B50F48006820F4F7
:1033A00040400D4908600846006840F480400860CD
:1033B00001200A4908600A49C1F898020A2001F070
:1033C0006DF90020054908600A2001F067F9002026
:1033D0000349C1F8980210BD000402409C8240429B
:1033E0000080404210B5022001F058F910480068F2
:1033F00020F440400E4908600846006840F48040D0
:10340000086000200B4908600B49C1F89C020A20A3
:1034100001F044F9012007490860052001F03EF958
:1034200001200549C1F89C020A2001F037F910BDBE
:1034300000040240988240420080404210B50024BF
:103440001148006820F440400F49086008460068B1
:1034500008600A2001F022F901200C4908600A20C6
:1034600001F01CF907E0601CC4B2FA2C03DDFFF781
:10347000B9FF012010BD05487C3800680028F2D152
:103480000249086000BFF5E700040240988240420C
:1034900010B500F001F810BD4AF6AA2001490860F5
:1034A000704700000030004070B505460E4600240D
:1034B00010E02A5D02F0010104F12602D0B200F012
:1034C00017F82A5D52105100621CD0B200F010F8BB
:1034D000601CC4B2B442ECDB00F001F870BD10B562
:1034E0000121252000F004F8142001F0D7F810BDC8
:1034F00070B506460D460024102000F0EEF8C820F6
:1035000001F0CCF8FFF748FF7820FFF711FFFFF735
:1035100095FF044604B110E03046FFF709FFFFF7BE
:103520008DFF044604B108E02846FFF701FFFFF7CE
:1035300085FF044604B100E000BFFFF753FFC82039
:1035400001F0ACF870BD000010B54FF4A06000F0C1
:1035500067F80121022000F0A5FBA82001F060F827
:103560004FF4E13001F08EF9FDF7CEF8FEF762FC82
:1035700000F0B2F9FDF750F8FFF7BEF8002000F0B8
:103580005FFB01200149087010BD0000AA00002067
:1035900002480349086000BFFEE700000400FA0586
:1035A0000CED00E07047000070B5002100230F22F1
:1035B000C4781CB3174C246804F4E064C4F5E064D8
:1035C000C4F30721C1F10404E3B20A4144789C40EA
:1035D000E1B28478144021430C07210E0E4C05788B
:1035E0006155047804F01F050124AC4005786D1185
:1035F000AD0005F1E025C5F8004109E0047804F0CC
:103600001F050124AC40054D0678761145F826408B
:1036100070BD00000CED00E000E400E080E100E09F
:1036200002490143024A1160704700000000FA0598
:103630000CED00E070B582240325FFF7ADFE2046B7
:10364000FFF776FEFFF7FAFE00B10EE02846FFF71F
:103650006FFEFFF7F3FE00B107E00020FFF768FE02
:10366000FFF7ECFE00B100E000BFFFF7BBFE70BD4E
:1036700070B5044682250126FFF78EFE2846FFF727
:1036800057FEFFF7DBFE00B110E03046FFF750FEBB
:10369000FFF7D4FE00B109E004F00101881CFFF738
:1036A00047FEFFF7CBFE00B100E000BFFFF79AFE38
:1036B00070BD70B50024FFF76FFEE1252846FFF7C7
:1036C00037FEFFF7BBFE0020FFF7FCFD0446FFF7C7
:1036D000D1FDFFF787FE204670BD70B50446FFF7A9
:1036E0005BFEE0252846FFF723FEFFF7A7FE00B1AB
:1036F00007E02046FFF71CFEFFF7A0FE00B100E048
:1037000000BFFFF76FFE70BD704700007CB5044638
:103710000D46012C06D0022C0AD0032C0ED0042C0E
:1037200018D111E0144800900015ADF8040012E023
:10373000124800900015ADF804000CE0104800900D
:103740000220ADF8040006E00C4800900820ADF817
:10375000040000E07CBD00BF012D05D1BDF80410C0
:103760000098FFF78AFA04E0BDF804100098FFF70C
:1037700086FA00BFEEE70000000C02400010024095
:10378000000802402DE9F05F04460E46207800F064
:103790000107207800F00208207800F00409207862
:1037A00000F0080A207800F0100B002537B1012541
:1037B0002846FFF792FF012000F050FFB8F1000FFC
:1037C00006D002252846FFF788FF012000F046FFBB
:1037D000B9F1000F06D004252846FFF77EFF01202F
:1037E00000F03CFFBAF1000F06D008252846FFF78D
:1037F00074FF012000F032FFBBF1000F06D010254E
:103800002846FFF76AFF012000F028FFFFF751FF6D
:10381000A84202D00020BDE8F09F35B164223146B5
:103820000020FCF762FE6420F5E70020F3E72DE9B5
:10383000F05F04460E46207800F00107207800F083
:103840000208207800F00409207800F0080A2078A7
:1038500000F0100B002537B101252846FFF73DFF8A
:10386000012000F0FBFEB8F1000F06D0022528462B
:10387000FFF733FF012000F0F1FEB9F1000F06D091
:1038800004252846FFF729FF012000F0E7FEBAF1E2
:10389000000F06D008252846FFF71FFF012000F083
:1038A000DDFEBBF1000F06D010252846FFF715FFFF
:1038B000012000F0D3FEFFF7FCFEA84202D000205A
:1038C000BDE8F09F2DB1642231460020FCF75BFE7D
:1038D000F6E70020F4E700001CB501210D2000F000
:1038E000E1F95420009000208DF8040001208DF8AB
:1038F000060003208DF8050000208DF807006946BA
:103900000F48FFF746F94FF4A050009069460D4864
:10391000FFF73FF94FF44070009001208DF8070049
:1039200069460848FFF735F969460748FFF731F956
:103930004FF40040009069460148FFF72AF91CBD8A
:10394000000C024000000240000802402DE9F04750
:1039500040212748FFF788F9054610212448FFF742
:1039600083F9064604212248FFF77EF907464FF403
:1039700080512048FFF778F980464FF480611D4858
:10398000FFF772F981461C48007818B9002501201C
:10399000194908701948007818B9002601201749FC
:1039A00008701748007818B90027012014490870DA
:1039B0001448007820B94FF0000801201149087020
:1039C0001148007820B94FF0000901200E49087015
:1039D00045F0E00040EA460040EA870040EAC800BF
:1039E00040EA0910C043C4B22046BDE8F087000099
:1039F000000C024000000240A5000020A6000020AC
:103A0000A7000020A8000020A90000202DE9F04711
:103A10004FF400717748FFF727F904464FF480719F
:103A20007448FFF721F905464FF400717248FFF71B
:103A30001BF906464FF480716F48FFF715F90746EA
:103A40004FF400416D48FFF70FF9804644F0E00065
:103A500040EA450040EA860040EAC70040EA081014
:103A6000C04300F0FF094FF400716248FFF7FCF813
:103A700063490978884216D04FF400715D48FFF71A
:103A8000F3F880B91E2000F0E9FD4FF400715948A9
:103A9000FFF7EAF838B90120FFF71FFE012000F018
:103AA000DDFDFFF7C7FD4FF480715248FFF7DCF8EA
:103AB00054490978884216D04FF480714D48FFF779
:103AC000D3F880B91E2000F0C9FD4FF48071494839
:103AD000FFF7CAF838B90220FFF7FFFD012000F018
:103AE000BDFDFFF7A7FD4FF400714348FFF7BCF899
:103AF00045490978884216D04FF400713E48FFF7D7
:103B0000B3F880B91E2000F0A9FD4FF400713A48C7
:103B1000FFF7AAF838B90420FFF7DFFD012000F015
:103B20009DFDFFF787FD4FF480713348FFF79CF848
:103B300036490978884216D04FF480712E48FFF735
:103B400093F880B91E2000F089FD4FF480712A4857
:103B5000FFF78AF838B90820FFF7BFFD012000F011
:103B60007DFDFFF767FD4FF400412448FFF77CF827
:103B700027490978884216D04FF400411F48FFF7C3
:103B800073F880B91E2000F069FD4FF400411B4816
:103B9000FFF76AF838B91020FFF79FFD012000F009
:103BA0005DFDFFF747FD4FF400711248FFF75CF829
:103BB000134908704FF480710E48FFF755F811490A
:103BC00008704FF400710C48FFF74EF80E4908706A
:103BD0004FF480710848FFF747F80C4908704FF41C
:103BE00000410648FFF740F8094908704846BDE81B
:103BF000F08700000000024000080240000C024074
:103C0000A0000020A1000020A2000020A3000020AE
:103C1000A400002070B504460D46052C00DC04B954
:103C200070BD601EC4B20121A140C8B2FFF755FDAE
:103C3000012000F013FD2846FFF71AFD00BFEFE753
:103C40002DE9F047044604F00105C4F34006C4F32F
:103C50008007C4F3C008C4F3001929460120FFF708
:103C6000D9FF012000F0FAFC31460220FFF7D2FF15
:103C7000012000F0F3FC39460320FFF7CBFF0120C1
:103C800000F0ECFC41460420FFF7C4FF012000F0E7
:103C9000E5FC49460520FFF7BDFF012000F0DEFCF2
:103CA000BDE8F08729B1064A12680243044B1A6046
:103CB00004E0034A12688243014B1A607047000017
:103CC0003038024029B1064A12680243044B1A6098
:103CD00004E0034A12688243014B1A6070470000F7
:103CE00044380240F0B500210022002402250026BD
:103CF0000223324F3F6807F00C0121B1042905D09F
:103D0000082937D105E02E4F076036E02D4F0760B8
:103D100033E02A4F3F1F3F68C7F38056274F3F1FAE
:103D20003F6807F03F036EB1264FB7FBF3F7DFF8AC
:103D30008CC0ACF1040CDCF800C0CCF3881C07FB91
:103D40000CF40CE01E4FB7FBF3F7DFF870C0ACF1DA
:103D5000040CDCF800C0CCF3881C07FB0CF4174FF4
:103D60003F1F3F68C7F301477F1C7D00B4FBF5F799
:103D7000076002E0124F076000BF00BF0F4F3F68AF
:103D800007F0F0010909104F7A5C0768D7404760D7
:103D90000A4F3F6807F4E051890A0B4F7A5C476885
:103DA000D7408760054F3F6807F46041490B064FD5
:103DB0007A5C4768D740C760F0BD00000838024011
:103DC0000024F40000127A000701002001461C487C
:103DD000814201D2002070471A48814201D2082056
:103DE000F9E71948814201D21020F4E717488142CF
:103DF00001D21820EFE71648814201D22020EAE7DD
:103E00001448814201D22820E5E71348814201D2BB
:103E10003020E0E71148814201D23820DBE710482A
:103E2000814201D24020D6E70E48814201D248208B
:103E3000D1E70D48814201D25020CCE75820CAE793
:103E4000004000080080000800C0000800000108D1
:103E5000000002080000040800000608000008082E
:103E600000000A0800000C0800000E0830B50346E8
:103E70000C461546002206E0184600F007F844F804
:103E800022001B1D521CAA42F6D330BD0146086811
:103E9000704700002DE9F04704460E4617464FF0E4
:103EA00009080025A946B4F1006F02D304F003000D
:103EB00008B1BDE8F087FEF749FE0020FEF794FD4B
:103EC000254604EB87091948854218D214E0284694
:103ED000FFF7DCFF401C70B1F120FEF77FFD2846A4
:103EE000FFF774FF82460221FEF790FD8046B8F18D
:103EF000090F01D002E02D1D4D45E8D300BFB8F1F8
:103F0000090F0CD108E020463168FEF7F7FD0928BB
:103F100000D003E0241D361D4C45F4D300BF012022
:103F2000FEF762FDFEF7E0FD00BFC2E70000FF1FE5
:103F30007047000030B500228B071C0F0F2303FAD7
:103F400004F20B4B8C1053F824309343084C8D1023
:103F500044F8253023468C1053F824308C07240F66
:103F600000FA04F42343024C8D1044F8253030BD90
:103F7000083801407CB504460D46012C06D0022CC1
:103F80000AD0032C0ED0042C18D111E01448009054
:103F90000220ADF8040012E0114800900120ADF8B5
:103FA00004000CE00F4800904015ADF8040006E056
:103FB0000C4800908015ADF8040000E07CBD00BF07
:103FC000012D05D1BDF804100098FEF758FE04E05D
:103FD000BDF804100098FEF750FE00BFEEE70000A9
:103FE00000100240000402400CB500200190009037
:103FF0003448006840F480303249086000BF3148DE
:10400000006800F4003000900198401C0190009876
:1040100018B90198B0F5A04FF1D12A48006800F412
:10402000003010B10120009001E0002000900098C5
:10403000012846D123484030006840F08050214993
:10404000403108602048006840F440401E49086044
:104050001C48083000681B490831086008460068A1
:1040600040F4004008600846006840F4A050086032
:104070001648091F0860081F006840F08070091F7B
:10408000086000BF0F48006800F000700028F9D0F9
:1040900040F205700E4908600A480830006820F0B8
:1040A00003000849083108600846006840F0020033
:1040B000086000BF03480830006800F00C000828C2
:1040C000F8D10CBD00380240007000400854400791
:1040D000003C0240042808D14FF0E021096941F07A
:1040E00004014FF0E022116107E04FF0E02109697F
:1040F00021F004014FF0E022116170477047000089
:1041000010B51548006840F4700013490860134862
:10411000006840F001001149086000200F49083193
:1041200008600E4800680E4908400C4908600D48B8
:10413000091D0860081F006820F48020091F08601E
:10414000002006490C310860FFF74EFF4FF0006079
:1041500001498039086010BD88ED00E00038024058
:10416000FFFFF6FE1030002410B50121054800F0D5
:1041700010F8012801D1044908700121014800F01C
:1041800005F810BD00040040AB000020CA430282C5
:10419000704730B50246002000230024158A05EA46
:1041A0000103958905EA010413B10CB1012000E077
:1041B000002030BD70B504460D46FFF727FC00B265
:1041C0001E490880FFF7C2FB00B21D490880012C80
:1041D00010D11C48B0F900001849B1F9001088420C
:1041E00008D11948B0F900001549B1F9001088420A
:1041F00000D170BD1148B0F9000012490880104884
:10420000B0F900001049088002260C4800780F49D8
:1042100008700B48007848702A463146312000F07B
:1042200017F90648B0F90000064908800448B0F9BB
:1042300000000549088000BFDBE700009C02002069
:104240009E020020A0020020A2020020B44600200E
:10425000002005E04FF6FF710B4A22F81010401CB9
:104260001428F7DB0020094908700949087009493A
:104270000870094908600949087009490880094916
:10428000088009490880704734570020AE0000209C
:10429000AC000020AD000020B0000020B4000020E1
:1042A000B6000020B8000020BA0000205E4909884E
:1042B00001F0200121B15C49091D0988C8B200E064
:1042C00070475A4909780A297BD2DFE801F00517BF
:1042D000232F353B4E52616D55280ED10121544A92
:1042E0001170544A11800021534A118001214F4A14
:1042F000117052490988524A118063E0AA2803D1FB
:1043000002214A4A117004E00021494A1170474ACB
:10431000117057E0BB2803D10321444A117004E017
:104320000021434A1170414A11704BE004213F4A79
:1043300011704149088045E005213C4A11703E4911
:1043400008803FE00621394A11703B49098841EA5B
:104350000021394A11800021364A118036490988E6
:1043600011B90821314A11702CE007212F4A117030
:1043700000BF30490988491C2E4A1180114609881E
:104380002D4A1288914202DB0821284A117019E057
:104390000D2805D00021264A1170244A117002E030
:1043A0000921224A11700DE00A2806D00021204A76
:1043B00011701E4A117003E003E00A211B4A1170BC
:1043C00000E000BF00BF1A49097881B11B490A68A3
:1043D0000968491C194B19601A498854194609681B
:1043E00044F20802914202D300211A4611600F499B
:1043F00009780A2915D112490988134A134B1B78E9
:1044000022F8131011490978491C142291FBF2F388
:1044100002FB13110D4A11700021054A1170034A65
:10442000117000BF4CE7000000140140AE000020F6
:10443000B4000020BA000020B8000020B000002026
:10444000B6000020AC06002034570020AC0000204D
:104450002DE9F04781460C461646274626B1A1B203
:104460001048FEF7A2FD7F000F4B3A460D49484623
:10447000FDF7DAF9804640210C4800F019F80025D4
:104480000CE00948415D094800F0C4F800BF402134
:10449000064800F022F80128F9D16D1C4545F0DBF3
:1044A000BDE8F087B4460020B44E0020001401405F
:1044B00001F40072B2F5007F00D100BFCA43028050
:1044C000704721B1828942F40052828104E08289DE
:1044D0004DF6FF731A408281704702460020B1F505
:1044E000007F00D100BF13880B400BB1012000E01A
:1044F00000207047F0B50346002400260025002068
:1045000040F66A17B94200D100BF1846C1F3421401
:1045100001F01F06012707FA06F5012C01D10C3026
:1045200004E0022C01D1103000E014301AB1076809
:104530002F43076002E00768AF430760F0BD00004B
:104540002DE9FF4705460E460024A14600BFA046C0
:10455000B08900B100BF2C8A24F44054F088044391
:104560002C82AC8941F20C608443B08831890843C5
:10457000718908430443AC81AC8A24F44074B08947
:104580000443AC826846FFF7ADFB2048854202D069
:104590001F48854202D1DDF80C9001E0DDF808905B
:1045A000A88900F4004040B109EBC90000EB0910F4
:1045B00031684900B0FBF1F707E009EBC90000EBF7
:1045C000091031688900B0FBF1F76420B7FBF0F007
:1045D00004012009642101FB1078A88900F400403F
:1045E00040B1322000EBC800B0FBF1F000F0070052
:1045F000044308E0322000EB08106421B0FBF1F026
:1046000000F00F0004432C81BDE8FF87001001403B
:1046100000140140C1F308028280704700BFFEE72A
:1046200010B504466FF00400FFF754FDE11704EBEA
:104630005171C1F3C701074A11701046007800EBB1
:104640004001C1EBC0104FF6FF7101EAC000024902
:10465000088010BD9C0000209E00002070B504461C
:104660004FF4077094FBF0F0C6B24FF4077094FB60
:10467000F0F100FB114085B204B970BD05E04FF4C4
:10468000077000F031F8701EC6B2002EF7D115B1D8
:10469000284600F029F800BFEFE700000146114A64
:1046A00012784A434FF0E0235A6100229A611A4679
:1046B000126942F001021A6100BF4FF0E022106956
:1046C00000F001021AB100F48032002AF5D04FF058
:1046D000E022126922F001024FF0E0231A61002269
:1046E0009A6170479C0000200146114A12884A4393
:1046F0004FF0E0235A6100229A611A46126942F093
:1047000001021A6100BF4FF0E022106900F00102BF
:104710001AB100F48032002AF5D04FF0E02212697D
:1047200022F001024FF0E0231A6100229A617047E3
:104730009E00002010B50446282221460148FFF7BC
:1047400095FB10BD0000010810B504462822214643
:104750000148FFF79FFB10BD0000010800B5A9B09C
:104760006846FFF7E7FF4FF0FF30CDF8820068465C
:10477000FFF7EAFF0A20FFF771FF29B000BD000034
:10478000FEF7E2FEFEF79EFB0024FDF7FDFAFDF7C3
:10479000FBFA01212948FDF7E3F902212748FDF73B
:1047A000DFF91F27A04600250CE0681CC2B239467D
:1047B0000420FDF701FE681CC2B241460520FDF74A
:1047C000FBFD6D1C042DF0DBFDF7D0F800260CE09E
:1047D000642094FBF0F100FB114008B9FEF758FE8D
:1047E000641C3220FFF75AFF761CB6F57A7FEFDBA8
:1047F0000024FDF7BBF81FE03220FFF74FFF6420D5
:1048000094FBF0F100FB114008B9FEF741FEFBF705
:1048100099FFFDF729F80A480078012800D10BE03C
:10482000B4F57A7F06DB01210846FFF7C3FCFDF7EC
:10483000ABFA0024641C00BFDEE70000FF7F20000D
:10484000840000200D48006840F480200B49086077
:104850000A481038006840F0100008491039086014
:10486000032001218140064A430942F8231000BF7A
:10487000BFF34F8FBFF36F8F7047000024ED00E050
:1048800000E200E010B588B0044601210420FFF7E3
:1048900009FA01212020FFF715FA082206212548F0
:1048A000FEF7BFF9082207212248FEF7BAF9C02017
:1048B000069002208DF81C008DF81D0000208DF858
:1048C0001E0001208DF81F0006A91A48FEF761F9A5
:1048D00002940020ADF80C00ADF80E00ADF8100009
:1048E000ADF814000C20ADF8120002A91248FFF731
:1048F00027FE01211048FFF7E4FD40210E48FFF795
:10490000D7FD012240F225510B48FFF7F3FD472068
:104910008DF8040002208DF8050003208DF80600B4
:1049200001208DF8070001A8FEF73EFEFFF790FC7E
:1049300008B010BD00080240001401404FF0407064
:10494000E1EE100A704700006849000800000020EE
:10495000AC020000C4010008D84A0008AC020020E4
:104960006C7D000020020008111214801801323002
:104970003234303730323131343730307A68616F29
:10498000796F6E670011104A6948654D736F383052
:1049900030305831306720002E313466643663661B
:1049A0006136EFBC9A63616E207265616420616C50
:1049B0006C206368616E6E656C732074656D7065E4
:1049C0007261747572652E7A0101011A12081B0852
:1049D0000603180A01080602080603080809101051
:1049E000070806060806050806040A08020A071E44
:1049F0000A07010A07092014030A08030A07070C1B
:104A000007060C07050C07040C48403C0301056B26
:104A10002C02030404193D92091808323032322D59
:104A20003031033D2030303A0311298B1BF90C77CC
:104A3000190932021B210D0C3132034B0D0E0C2AC9
:104A400004514A0F24295E1A390C29C432062A71EE
:104A50000C3132075AB52432155AE51832204B432F
:104A6000104832215A5B0C32225A5D0C32234BB96A
:104A700011302A29784A12182A3060290C19192A6B
:104A80003154590C32325AFD2432334B15139032C3
:104A9000342A850C312A4054590C2A41B44A140C4A
:104AA00032425AC10C32434B59150C2A4818590C42
:104AB00032505AF50C32C14B9D166C32E05AB10C93
:104AC00032E15AC90C32E31AD10C293032E44BAD31
:084AD000171801101AFF018103
:040000050800018965
:00000001FF
